:10000000830100308A0004282030840030300F2023
:1000100083010A128A117D2A04068001840A0406DB
:10002000031900340C2882070F34003400340034E4
:100030000F340034003400340F340F3400340034F3
:100040000F340F340F3400340F340F340F340F34A7
:10005000003400340034F03400340034F034F03430
:100060000034F034F034F034F034F034F034F03460
:100070008207F034003400340034F03400340034AB
:100080000034F034F03400340034F034F034F03420
:100090000034F034F034F034F03400340034003400
:1000A0000F34003400340F340F3400340F340F3465
:1000B0000F340F340F340F340F3482070834803478
:1000C00040342034103401348207103401340234B7
:1000D00004340834803482070F34F03400340034A0
:1000E0008207003400340F34F034820700340034C7
:1000F000F0340F348207F0340F34003400348207B8
:10010000883444342234113482071F3401340134DA
:1001100001348207113400340034003482079F34E4
:10012000093409349F348207F93490349034F93417
:1001300082070034603460340034820700340634AF
:0E014000063400348207FE34FD34FB34F734FD
:10043A00831203132D08A1002E08A200A301A40110
:10044A00A001A00A080083120313A008031D312A81
:10045A00AD01AD0AAE011D226D30F4004E30F5003B
:10046A00C630F6004130F7002108F0002208F100FA
:10047A002308F2002408F3000A128A11C3270A1279
:10048A008A113930F4003030F500F601F7017408AA
:10049A007007F8007108F90075080318750FF90755
:1004AA007208FA0076080318760FFA077308FB0039
:1004BA0077080318770FFB077808A1007908A200CC
:1004CA007A08A3007B08A400F1002308F0007F301B
:1004DA00F105080083120313AD000430AE00533057
:1004EA00AF00AF0B762AAE0B742AAD0B722A080046
:1004FA0083160313860188018701FF308312870060
:10050A0086018801AC0100308A002C08A2200A1258
:10051A008A118700AB010130F0002B08F100F10AC3
:10052A00982A0310F00DF10B962A7008880064309F
:10053A006F22AB0A08302B02031C902A8801AB01F8
:10054A000130F0002B08F100F10AAD2A0310F00D7A
:10055A00F10BAB2A7008860064306F22AB0A0830B0
:10056A002B02031CA52A8601AC0A04302C02031CA8
:10057A00882A5030A700AC0100308A002C08A2203B
:10058A000A128A118700AB010130F0002B08F10032
:10059A00F10AD12A0310F00DF10BCF2A7008880056
:1005AA0027086F22AB0A04302B02031CC92AAB01AD
:1005BA008030F0002B08F100F10AE52A0310F00C54
:1005CA00F10BE32A7008880027086F22AB0A04306F
:1005DA002B02031CDD2A8801AB010130F0002B0835
:1005EA00F100F10AFA2A0310F00DF10BF82A70084B
:1005FA00860027086F22AB0A04302B02031CF22A5A
:10060A00AB018030F0002B08F100F10A0E2B031029
:10061A00F00CF10B0C2B7008860027086F22AB0A2E
:10062A0004302B02031C062B8601AC0A04302C0270
:10063A00031CC12AAA01AC0100308A002C08A2209E
:10064A00870000308A002C088420880000308A0045
:10065A002C088920860001300A128A116F2286012D
:10066A008801AC0A04302C02031C212BAA0AC830C8
:10067A002A02031C202BA901AA01AC0100308A001E
:10068A002C08A220870000308A002C088E208800BF
:10069A0000308A002C089320860001300A128A1141
:1006AA006F2286018801AC0A04302C02031C432BFA
:1006BA00AA0AC8302A02031C422BAA01AC01003044
:1006CA008A002C08A220870000308A002C08982073
:1006DA00880000308A002C089D20860001300A120A
:1006EA008A116F2286018801AC0A04302C02031C8D
:1006FA00642BAA0AC8302A02031C632BA90A0230F7
:10070A002902031C412BA901AB01AA01AC012C0847
:10071A002B06031D982B00308A002C08A220870084
:10072A00FF308800860001300A128A116F22880180
:10073A008601AC0A04302C02031C8C2BAA0A28302E
:10074A002A02031C8B2BAB0A04302B02031C8A2BB4
:10075A000430AB00AA010430AC002C082B06031DA0
:10076A00BE2B00308A002C03A2208700FF308800AD
:10077A00860001300A128A116F2288018601AC0BA9
:10078A00B22BAA0A28302A02031CB02BAB0BAF2BC0
:10079A00A90A02302902031C892BA901AB01AA016B
:1007AA00AC012C082B02031CE22B00308A002C0817
:1007BA00A2208700FF308800860001300A128A11C1
:1007CA006F2288018601AC0A04302C02031CD62B46
:1007DA00AA0A28302A02031CD52BAB0A04302B02A2
:1007EA00031CD42B0430AB00AA010430AC002C0843
:0607FA002B02031C082C79
:1008000000308A002C03A2208700FF308800860079
:1008100001300A128A116F2288018601AC0BFC2B71
:10082000AA0A28302A02031CFA2BAB0BF92BA90ABF
:1008300002302902031CD32BA901AB01AA01AC0190
:1008400000308A002C08A220870000308A002B0884
:100850006B20880000308A002B0870208600013051
:100860000A128A116F22AC0A04302C02031C202CBD
:10087000AA0A28302A02031C1F2C88018601AB0A11
:1008800004302B02031C1E2CAB01AA01AC0100306A
:100890008A002C08A220870000308A002B087520CF
:1008A000880000308A002B087A20860001300A1266
:1008B0008A116F22AC0A04302C02031C472CAA0AAE
:1008C00028302A02031C462C88018601AB0A04301A
:1008D0002B02031C452CA90A02302902031C1D2CE3
:1008E000A901AB01AA01AC0100308A002C08A220AA
:1008F000870000308A002B087F20880000308A00A3
:100900002B087F20860001300A128A116F22AC0A60
:1009100004302C02031C742CAA0A28302A02031C5F
:10092000732C86018801AB0A04302B02031C722C45
:10093000AB01AA01AC0100308A002C08A22087007C
:1009400000308A002B08033C7F20880000308A009A
:100950002B08033C7F20860001300A128A116F2287
:10096000AC0A04302C02031C9B2CAA0A28302A0251
:10097000031C9A2C86018801AB0A04302B02031C4D
:10098000992CA90A02302902031C712C86018801C6
:10099000AB01AA01AC0100308A002C08A22087001C
:1009A00000308A002B086420880001300A128A1166
:1009B0006F22AC0A04302C02031CCB2CAA0A143080
:1009C0002A02031CCA2CAB0A06302B02031CC92CBA
:1009D0008801AB01AA01AC0100308A002C08A220DA
:1009E000870000308A002B085D20860001300A1243
:1009F0008A116F22AC0A04302C02031CEC2CAA0AC8
:100A000014302A02031CEB2CAB0A06302B02031C09
:100A1000EA2C860186018801AB01AA01AC010030F5
:100A20008A002C08A220870000308A002B0864204E
:100A3000880401300A128A116F22AC0A04302C0299
:100A4000031C0F2DAA0A14302A02031C0E2DAB0A18
:100A500006302B02031C0D2DAB01AA01AC010030A6
:100A60008A002C08A220870000308A002B085D2015
:100A7000860401300A128A116F22AC0A04302C025B
:100A8000031C2F2DAA0A14302A02031C2E2DAB0A98
:100A900006302B02031C2D2D86018801A901A90A0D
:100AA000AB01AA01AC0129082C020318672D003004
:100AB0008A002C08A220870000308A002B086420BE
:100AC000880401300A128A116F22AC0A532DAA0A37
:100AD00014302A02031C522DAB0A06302B02031CD1
:100AE000512D8801AB01AA01AC0129082C02031881
:100AF000892D00308A002C08A220870000308A004F
:100B00002B085D20860401300A128A116F22AC0A7C
:100B1000752DAA0A14302A02031C742DAB0A063064
:100B20002B02031C732D8601A90A05302902031C20
:100B3000502D6430A700AC0100308A002C08A220A0
:100B400087000F30880027080A128A116F22F030C0
:100B5000880027086F2288010F30860027086F223F
:100B6000F030860027086F22F030860027086F22B9
:100B70000F30860027086F228601F0308800270892
:100B80006F220F30880027086F22AC0A04302C0235
:100B9000031C9C2D6430A700AB01A901AA018601AA
:100BA00088010A128A11A320870000308A002908D0
:100BB0006B20880000308A002908702086000130F0
:100BC0000A128A116F228601880100308A000330E0
:100BD000A220870000308A0029087A208600003091
:100BE0008A0029087520880001300A128A116F22B4
:100BF000AA0A32302A02031CCF2DA90A0430290286
:100C0000031CCE2DA901AA01860188010A128A11AE
:100C1000A320870000308A00290875208800003052
:100C20008A0029087A20860001300A128A116F2270
:100C30008601880100308A000330A220870000303E
:100C40008A0029087020860000308A0029086B205D
:100C5000880001300A128A116F22AA0A32302A0251
:100C6000031C042EA90A04302902031C032EAB0A1C
:100C700004302B02A901031CCE2D0A128A1128224E
:100C80007008A5000A128A1128227008A600AA017D
:100C9000AC018601880100308A002C08A220870060
:100CA000250888002608860001300A128A116F2262
:100CB000AC0A04302C02031C492EAA0A64302A0212
:100CC000031C482EA90A0A302902031C3D2EA90143
:100CD000AA01AC018601880100308A002C08A220FC
:100CE000870000308A002908F0000310F00D03107F
:100CF000700D2C073820880000308A002908F00089
:100D00000310F00D0310700D2C0713208600013026
:100D10000A128A116F22AC0A04302C02031C6A2EBC
:100D2000AA0A28302A02031C692EA90A09302902BE
:100D3000031C682EAC01AA018601880100308A00DC
:100D40002C08A220870009308800903086000130EE
:100D50000A128A116F22AA0A96302A02031C9C2EBC
:100D6000AC0A04302C02031C9B2EAC01AA018601A4
:100D7000880100308A002C08033CA220870009303B
:100D800088009030860001300A128A116F22AA0A68
:100D900096302A02031CB72EAC0A04302C02031C26
:100DA000B62E0F30A900A801AB01AA0129082A021A
:100DB0000318092FAC012C082B02031CFE2E003057
:100DC0008A002C08A2200A128A1187000130F00044
:100DD0002808F100F10AEE2E0310F00DF10BEC2EB5
:100DE000700888008030F0002808F100F10AFA2E1F
:100DF0000310F00CF10BF82E7008860001306F2202
:100E000086018801AC0A04302C02031CDB2EAA0ADE
:100E1000D62EAB0A04302B02031CD52E0430AB00B7
:100E2000AA0129082A020318422F0430AC002C081A
:100E30002B02031C3A2F00308A002C03A2200A1236
:100E40008A1187000130F0002808F100F10A2A2FEA
:100E50000310F00DF10B282F700888008030F0008F
:100E60002808F100F10A362F0310F00CF10B342F93
:100E70007008860001306F2288018601AC0B172FA5
:100E8000AA0A112FAB0B102F2908F0000310F00D48
:100E90000310700D6F22A80A08302802031CD42EFC
:100EA0000730A80086018801AC0100308A002C08B8
:100EB000A2208700AB0100308A002B086420880044
:100EC00028080A128A116F22AB0A06302B02031C73
:100ED0005B2F880100308A002C08A2208700AB011C
:100EE00000308A002B085D20860028080A128A112B
:100EF0006F22AB0A06302B02031C702F8601AC0A4E
:100F000004302C02031C552F86018801AC010030EF
:100F10008A002C08033CA2208700AB0100308A0025
:100F20002B08053C6420880028080A128A116F22C9
:100F3000AB0A06302B02031C8E2F880100308A007A
:100F40002C08033CA2208700AB0100308A002B084C
:100F5000053C5D20860028080A128A116F22AB0A20
:100F600006302B02031CA52F8601AC0A04302C028C
:100F7000031C872F0530A8071E302802031C522FA0
:100F80000A128A11042884017008F8007108F90017
:100F90007208FA007308FB00F201F301F001F1019D
:100FA0000310FB0CFA0CF90CF80C031CE52F740869
:100FB000F00775080318750FF10776080318760F08
:100FC000F20777080318770FF307780879047A0493
:100FD0007B040319F12F0310F40DF50DF60DF70D39
:100FE000D02F84080319003473088000840372082A
:100FF000800084037108800084037008800000343E
:02400E0071FF40
:00000001FF
